 adcsdk

 Timestamp is 4fb05c6a (Mon May 14 13:14:18 2012)

 Preferred load address is 10000000

 Start         Length     Name                   Class
 0001:00000000 00000004H .CRT$XCA                CODE
 0001:00000004 00000004H .CRT$XCZ                CODE
 0001:00000008 00000004H .CRT$XIA                CODE
 0001:0000000c 00000004H .CRT$XIZ                CODE
 0001:00000010 00000004H .CRT$XPA                CODE
 0001:00000014 00000004H .CRT$XPZ                CODE
 0001:00000018 00000004H .CRT$XTA                CODE
 0001:0000001c 00000004H .CRT$XTZ                CODE
 0001:00000020 00000508H .rdata                  CODE
 0001:00000528 00000023H .rdata$debug            CODE
 0001:0000054c 00001140H .text                   CODE
 0001:0000168c 00000014H .xdata                  CODE
 0001:000016a0 00000014H .idata$2                CODE
 0001:000016b4 00000014H .idata$3                CODE
 0001:000016c8 0000005cH .idata$4                CODE
 0001:00001724 0000000cH .idata$6                CODE
 0001:00001730 0000008fH .edata                  CODE
 0002:00000000 0000005cH .idata$5                DATA
 0002:00000060 00000480H .data                   DATA
 0002:000004e0 00000014H .bss                    DATA
 0003:00000000 000000b8H .pdata                  DATA

  Address         Publics by Value              Rva+Base       Lib:Object

 0000:00000000       ___safe_se_handler_count   00000000     <absolute>
 0000:00000000       ___safe_se_handler_table   00000000     <absolute>
 0001:00000000       __xc_a                     10001000     corelib0:crt0init.obj
 0001:00000004       __xc_z                     10001004     corelib0:crt0init.obj
 0001:00000008       __xi_a                     10001008     corelib0:crt0init.obj
 0001:0000000c       __xi_z                     1000100c     corelib0:crt0init.obj
 0001:00000010       __xp_a                     10001010     corelib0:crt0init.obj
 0001:00000014       __xp_z                     10001014     corelib0:crt0init.obj
 0001:00000018       __xt_a                     10001018     corelib0:crt0init.obj
 0001:0000001c       __xt_z                     1000101c     corelib0:crt0init.obj
 0001:00000040       ??_C@_1FE@EJPJFDIN@?$AAA?$AAd?$AAc?$AAI?$AAn?$AAi?$AAt?$AA?5?$AA?3?$AA?5?$AAF?$AAa?$AAi?$AAl?$AAe?$AAd?$AA?5?$AAw?$AAh?$AAi?$AAl?$AAe?$AA?5?$AAc?$AAr?$AAe?$AAa?$AAt?$AAi?$AAn?$AAg?$AA?5@ 10001040     adcsdk_common_topaz_v1:adc_sdk.obj
 0001:00000094       ??_C@_1BE@FABCBOME@?$AAM?$AAU?$AAT?$AAE?$AAX?$AA_?$AAA?$AAD?$AAC?$AA?$AA@ 10001094     adcsdk_common_topaz_v1:adc_sdk.obj
 0001:000000a8       ??_C@_1GE@KIKLFFGF@?$AAA?$AAd?$AAc?$AAI?$AAn?$AAi?$AAt?$AA?5?$AA?3?$AA?5?$AAC?$AAo?$AAu?$AAl?$AAd?$AA?5?$AAn?$AAo?$AAt?$AA?5?$AAr?$AAe?$AAt?$AAr?$AAi?$AAe?$AAv?$AAe?$AA?5?$AAa?$AAn?$AA?5@ 100010a8     adcsdk_common_topaz_v1:adc_sdk.obj
 0001:0000010c       ??_C@_1CI@OHCJFJPM@?$AAE?$AAR?$AAR?$AAO?$AAR?$AA?3?$AA?5?$AA?$CF?$AAs?$AA?5?$AAl?$AAi?$AAn?$AAe?$AA?5?$AA?$CF?$AAd?$AA?3?$AA?5?$AA?$AA@ 1000110c     adcsdk_common_topaz_v1:adc_sdk.obj
 0001:00000138       ??_C@_1LG@FIFJKOCD@?$AAC?$AA?3?$AA?2?$AAW?$AAI?$AAN?$AAC?$AAE?$AAR?$AAO?$AAO?$AAT?$AAS?$AA?2?$AAT?$AAo?$AAp?$AAa?$AAz?$AA?2?$AAW?$AAI?$AAN?$AAC?$AAE?$AA6?$AA0?$AA0?$AA?2?$AAP?$AAL?$AAA@ 10001138     adcsdk_common_topaz_v1:adc_sdk.obj
 0001:000001f0       ??_C@_1M@EPBPGMBG@?$AAA?$AAD?$AAC?$AA1?$AA?3?$AA?$AA@ 100011f0     adcsdk_common_topaz_v1:adc_sdk.obj
 0001:00000200       ??_C@_1GO@HPGCNGJP@?$AAA?$AAd?$AAc?$AAG?$AAe?$AAt?$AAS?$AAa?$AAm?$AAp?$AAl?$AAe?$AAs?$AA?5?$AA?3?$AA?5?$AAF?$AAa?$AAi?$AAl?$AAe?$AAd?$AA?5?$AAw?$AAh?$AAi?$AAl?$AAe?$AA?5?$AAc?$AAo?$AAn@ 10001200     adcsdk_common_topaz_v1:adc_sdk.obj
 0001:00000270       ??_C@_1HO@CKCOPGMD@?$AAA?$AAd?$AAc?$AAG?$AAe?$AAt?$AAS?$AAa?$AAm?$AAp?$AAl?$AAe?$AAs?$AA?5?$AA?3?$AA?5?$AAF?$AAa?$AAi?$AAl?$AAe?$AAd?$AA?5?$AAw?$AAh?$AAi?$AAl?$AAe?$AA?5?$AAi?$AAs?$AAs@ 10001270     adcsdk_common_topaz_v1:adc_sdk.obj
 0001:000002f0       ??_C@_1HM@PFPOFNKH@?$AAF?$AAa?$AAi?$AAl?$AAe?$AAd?$AA?5?$AAw?$AAh?$AAi?$AAl?$AAe?$AA?5?$AAr?$AAe?$AAt?$AAr?$AAi?$AAe?$AAv?$AAi?$AAn?$AAg?$AA?5?$AAs?$AAa?$AAm?$AAp?$AAl?$AAe?$AAs?$AA?5@ 100012f0     adcsdk_common_topaz_v1:adc_sdk.obj
 0001:00000370       ??_C@_1IA@BJCLINLD@?$AAA?$AAd?$AAc?$AAG?$AAe?$AAt?$AAS?$AAa?$AAm?$AAp?$AAl?$AAe?$AAs?$AA?5?$AA?3?$AA?5?$AAF?$AAa?$AAi?$AAl?$AAe?$AAd?$AA?5?$AAw?$AAh?$AAi?$AAl?$AAe?$AA?5?$AAi?$AAs?$AAs@ 10001370     adcsdk_common_topaz_v1:adc_sdk.obj
 0001:000003f0       ??_C@_1HK@ILFFIHH@?$AAA?$AAd?$AAc?$AAG?$AAe?$AAt?$AAS?$AAa?$AAm?$AAp?$AAl?$AAe?$AAs?$AA?5?$AA?3?$AA?5?$AAF?$AAa?$AAi?$AAl?$AAe?$AAd?$AA?5?$AAw?$AAh?$AAi?$AAl?$AAe?$AA?5?$AAc?$AAo?$AAn@ 100013f0     adcsdk_common_topaz_v1:adc_sdk.obj
 0001:00000470       ??_C@_1FM@KBKJHKGI@?$AA?$CK?$AA?$CK?$AA?$CK?$AA?$CK?$AA?$CK?$AA?5?$AAD?$AAL?$AAL?$AA?5?$AAP?$AAR?$AAO?$AAC?$AAE?$AAS?$AAS?$AA?5?$AAD?$AAE?$AAT?$AAA?$AAC?$AAH?$AA?5?$AAF?$AAR?$AAO?$AAM?$AA?5?$AAA?$AAD@ 10001470     adcsdk_common_topaz_v1:adc_sdk.obj
 0001:000004d0       ??_C@_1FI@LAGBOELG@?$AA?$CK?$AA?$CK?$AA?$CK?$AA?$CK?$AA?$CK?$AA?5?$AAD?$AAL?$AAL?$AA?5?$AAP?$AAR?$AAO?$AAC?$AAE?$AAS?$AAS?$AA?5?$AAA?$AAT?$AAT?$AAA?$AAC?$AAH?$AA?5?$AAT?$AAO?$AA?5?$AAA?$AAD?$AAC?$AA?5@ 100014d0     adcsdk_common_topaz_v1:adc_sdk.obj
 0001:0000054c       AdcInit                    1000154c f   adcsdk_common_topaz_v1:adc_sdk.obj
 0001:00000694       AdcDeinit                  10001694 f   adcsdk_common_topaz_v1:adc_sdk.obj
 0001:000006f8       AdcConfigureChannel        100016f8 f   adcsdk_common_topaz_v1:adc_sdk.obj
 0001:000009c8       AdcGetSamples              100019c8 f   adcsdk_common_topaz_v1:adc_sdk.obj
 0001:00000d50       DllEntry                   10001d50 f   adcsdk_common_topaz_v1:adc_sdk.obj
 0001:00000e18       CloseHandle                10001e18 f   coredll:COREDLL.dll
 0001:00000e28       CreateMutexW               10001e28 f   coredll:COREDLL.dll
 0001:00000e38       NKDbgPrintfW               10001e38 f   coredll:COREDLL.dll
 0001:00000e48       CreateFileW                10001e48 f   coredll:COREDLL.dll
 0001:00000e58       ReleaseMutex               10001e58 f   coredll:COREDLL.dll
 0001:00000e68       DeviceIoControl            10001e68 f   coredll:COREDLL.dll
 0001:00000e78       WaitForSingleObject        10001e78 f   coredll:COREDLL.dll
 0001:00000e88       DisableThreadLibraryCalls  10001e88 f   coredll:COREDLL.dll
 0001:00000e98       RegisterDbgZones           10001e98 f   coredll:COREDLL.dll
 0001:00000ea8       _DllEntryCRTStartup        10001ea8 f   corelib0:pegdentry.obj
 0001:00000f18       exit                       10001f18 f   corelib0:cexit.obj
 0001:00001098       _exit                      10002098 f   corelib0:cexit.obj
 0001:000010bc       _cexit                     100020bc f   corelib0:cexit.obj
 0001:000010d8       _c_exit                    100020d8 f   corelib0:cexit.obj
 0001:000010f4       GetCurrentProcess          100020f4 f i corelib0:cexit.obj
 0001:0000110c       _initterm                  1000210c f   corelib0:crt0dat.obj
 0001:00001160       _cinit                     10002160 f   corelib0:crt0dat.obj
 0001:00001194       __security_init_cookie     10002194 f   corelib0:seccinit.obj
 0001:00001264       _onexit                    10002264 f   corelib0:onexit.obj
 0001:00001568       atexit                     10002568 f   corelib0:onexit.obj
 0001:000015bc       free                       100025bc f   corelib1:COREDLL.dll
 0001:000015cc       __security_gen_cookie2     100025cc f   corelib1:COREDLL.dll
 0001:000015dc       __C_specific_handler       100025dc f   corelib1:COREDLL.dll
 0001:000015ec       malloc                     100025ec f   corelib1:COREDLL.dll
 0001:000015fc       realloc                    100025fc f   corelib1:COREDLL.dll
 0001:0000160c       _msize                     1000260c f   corelib1:COREDLL.dll
 0001:0000161c       DeleteCriticalSection      1000261c f   coredll:COREDLL.dll
 0001:0000162c       InterlockedExchange        1000262c f   coredll:COREDLL.dll
 0001:0000163c       TerminateProcess           1000263c f   coredll:COREDLL.dll
 0001:0000164c       EnterCriticalSection       1000264c f   coredll:COREDLL.dll
 0001:0000165c       InterlockedCompareExchange 1000265c f   coredll:COREDLL.dll
 0001:0000166c       InitializeCriticalSection  1000266c f   coredll:COREDLL.dll
 0001:0000167c       LeaveCriticalSection       1000267c f   coredll:COREDLL.dll
 0001:000016a0       __IMPORT_DESCRIPTOR_COREDLL 100026a0     coredll:COREDLL.dll
 0001:000016b4       __NULL_IMPORT_DESCRIPTOR   100026b4     coredll:COREDLL.dll
 0002:00000000       __imp_CloseHandle          10003000     coredll:COREDLL.dll
 0002:00000004       __imp_CreateMutexW         10003004     coredll:COREDLL.dll
 0002:00000008       __imp_NKDbgPrintfW         10003008     coredll:COREDLL.dll
 0002:0000000c       __imp_CreateFileW          1000300c     coredll:COREDLL.dll
 0002:00000010       __imp_ReleaseMutex         10003010     coredll:COREDLL.dll
 0002:00000014       __imp_DeviceIoControl      10003014     coredll:COREDLL.dll
 0002:00000018       __imp_WaitForSingleObject  10003018     coredll:COREDLL.dll
 0002:0000001c       __imp_DisableThreadLibraryCalls 1000301c     coredll:COREDLL.dll
 0002:00000020       __imp_RegisterDbgZones     10003020     coredll:COREDLL.dll
 0002:00000024       __imp_free                 10003024     corelib1:COREDLL.dll
 0002:00000028       __imp___security_gen_cookie2 10003028     corelib1:COREDLL.dll
 0002:0000002c       __imp___C_specific_handler 1000302c     corelib1:COREDLL.dll
 0002:00000030       __imp_malloc               10003030     corelib1:COREDLL.dll
 0002:00000034       __imp_realloc              10003034     corelib1:COREDLL.dll
 0002:00000038       __imp__msize               10003038     corelib1:COREDLL.dll
 0002:0000003c       __imp_DeleteCriticalSection 1000303c     coredll:COREDLL.dll
 0002:00000040       __imp_InterlockedExchange  10003040     coredll:COREDLL.dll
 0002:00000044       __imp_TerminateProcess     10003044     coredll:COREDLL.dll
 0002:00000048       __imp_EnterCriticalSection 10003048     coredll:COREDLL.dll
 0002:0000004c       __imp_InterlockedCompareExchange 1000304c     coredll:COREDLL.dll
 0002:00000050       __imp_InitializeCriticalSection 10003050     coredll:COREDLL.dll
 0002:00000054       __imp_LeaveCriticalSection 10003054     coredll:COREDLL.dll
 0002:00000058       \177COREDLL_NULL_THUNK_DATA 10003058     coredll:COREDLL.dll
 0002:00000060       dpCurSettings              10003060     adcsdk_common_topaz_v1:adc_sdk.obj
 0002:000004d8       __security_cookie          100034d8     corelib0:seccinit.obj
 0002:000004dc       __security_cookie_complement 100034dc     corelib0:seccinit.obj
 0002:000004e4       _exitflag                  100034e4     corelib0:cexit.obj
 0002:000004e8       __onexitend                100034e8     <common>
 0002:000004ec       __onexitbegin              100034ec     <common>
 0002:000004f0       g_pcsExit                  100034f0     <common>

 entry point at        0001:00000ea8

 Static symbols

 0001:0000092c       ?ValidateID@@YAHW4CHAN_ID@@@Z 1000192c f   adcsdk_common_topaz_v1:adc_sdk.obj
 0001:00000970       ?ValidateRef@@YAHW4POS_REF@@@Z 10001970 f   adcsdk_common_topaz_v1:adc_sdk.obj
 0001:00000f3c       doexit                     10001f3c f   corelib0:cexit.obj
 0001:000012c0       lockexit                   100022c0 f   corelib0:onexit.obj
 0001:0000135c       unlockexit                 1000235c f   corelib0:onexit.obj
 0001:00001388       _onexit_nolock             10002388 f   corelib0:onexit.obj
